:0200000480007A
:100000009710000093800000171100001301810178
:1000100083A10000139211009392F1001393F10158
:100020009393010013940101232031002322410006
:10003000232451002326610023287100232A8100F4
:1000400097100000938040FC17110000130101FF7E
:1000500003A40000931414001315F4009315F40185
:10006000131604009316040123208100232291001B
:100070002324A1002326B1002328C100232AD10074
:1000800097100000938080F817110000130181FC85
:1000900083A60000139716009397F6001398F601B5
:1000A00093980600139906012320D1002322E10032
:1000B0002324F1002326010123281101232A2101F1
:1000C000171600001306C6F497160000938606FA6A
:1000D0000329060093191900131AF900931AF9015C
:1000E000131B0900931B090123A0260123A236013B
:1000F00023A4460123A6560123A8660123AA76015C
:1001000017160000130606F197160000938686F76F
:10011000832B0600139C1B00939CFB00139DFB018B
:10012000939D0B00139E0B0123A0760123A2860151
:1001300023A4960123A6A60123A8B60123AAC601DB
:10014000171D0000130D4DED971D0000938D0DF54B
:10015000032E0D00931E1E00139F1E00931F1F00F1
:1001600093901F00139110009311110023A0CD0153
:1001700023A2DD0123A4ED0123A6FD0123A81D0078
:1001800023AA2D0023AC3D0097100000938000E9C6
:1001900017110000130141F283A200001390120016
:1001A0002320010097100000938080E717110000C2
:1001B0001301C1F083A200001390120093121000EB
:1001C000232001002322510017150000130585E5A7
:1001D00097150000938505EF370610F01306C6F259
:1001E0006306B5028326C5002320D600832685003A
:1001F0002320D600832645002320D6008326050031
:100200002320D600130505016FF09FFD370510F080
:10021000130505F223200500000000000000000087
:0402200000000000DA
:101000000000000001000000FFFFFFFFFFFFFF7F67
:101010000000008010EFCDAB7856341298BADCFE99
:10102000FFFFFFFFFFFFFFFFFFFFFFFFFFFFFFFFD0
:10103000FFFFFFFFFFFFFFFFFFFFFFFFFFFFFFFFC0
:10104000FFFFFFFFFFFFFFFFFFFFFFFFFFFFFFFFB0
:10105000FFFFFFFFFFFFFFFFFFFFFFFFFFFFFFFFA0
:10106000FFFFFFFFFFFFFFFFFFFFFFFFFFFFFFFF90
:10107000FFFFFFFFFFFFFFFFFFFFFFFFFFFFFFFF80
:10108000FFFFFFFFFFFFFFFFFFFFFFFFFFFFFFFF70
:10109000FFFFFFFFFFFFFFFFFFFFFFFFFFFFFFFF60
:1010A000FFFFFFFFFFFFFFFFFFFFFFFFFFFFFFFF50
:1010B000FFFFFFFFFFFFFFFFFFFFFFFFFFFFFFFF40
:040000058000000077
:00000001FF
